:10000000180800105501000000000000000000006A
:10001000C1020000C1020000C10200000000000097
:10002000000000000000000000000000C10200000D
:10003000C102000000000000C1020000C102000077
:10004000C1020000C1020000C1020000C1020000A4
:10005000C1020000C1020000C1020000C102000094
:10006000C1020000C1020000C1020000C102000084
:10007000C1020000C1020000C1020000C102000074
:10008000C1020000C1020000C1020000C102000064
:10009000C1020000C1020000C1020000C102000054
:1000A000C1020000C1020000C1020000C102000044
:1000B000C1020000C1020000C1020000C102000034
:1000C000C102000070B582B000F0C4F91D4D1E4E93
:1000D00043F6FF741D4B9D422ADDB5422BDCA5F58E
:1000E0009C45203D284600F035FB194B00215869FE
:1000F00040F480225A6101910198A04205DC019BE5
:100100005A1C01920199A142F9DD114B0021586955
:1001100020F480225A6101910198A042DADC019B0F
:100120005A1C01920199A142F9DD084B9D42D4DC91
:10013000044D2846D7E7A5F54235A5F5A86528461C
:10014000D1E700BF00E1F5057FC3C9013F420F00C1
:1001500020C00920684620F007018D46F1B500F067
:10016000B1F84F484F49884235D04F4CA14232D266
:10017000024652F8046B0B46CD4343F8046B6519F5
:10018000A342C5F3810526D29DB1012D0BD0022DCE
:1001900005D0156800F108021D6001F1080352F84E
:1001A000040B43F8040B52F8041B43F8041BA3424E
:1001B00011D296465EF8047B5668D568DEF80400D6
:1001C0009C464CF8047B5E60CCF80400DD60103384
:1001D0001032A342EDD335483549884234D0354CEE
:1001E000A14231D2024652F8046B0B46CD4343F88C
:1001F000046B6519A342C5F3810525D29DB1012D7C
:100200000BD0022D05D0156800F108021D6001F128
:10021000080352F8040B43F8040B52F8041B43F88C
:10022000041BA34210D294465CF8047B5668D56840
:10023000DCF80400194641F8047B5E604860DD602C
:1002400010331032A342EED31B491C48814221D205
:1002500000220B46CC4343F8042B04198342C4F319
:10026000810417D264B1012C06D0022C1CBF1A6085
:1002700001F1080343F8042B43F8042B834209D20D
:100280009E464EF8042B5A60CEF80420DA601033F4
:100290008342F5D3FFF716FFBDE8F140854670476E
:1002A00018090000000000100C00001018090000E0
:1002B00000000010000000100C00001018000010DA
:1002C000FEE700BF3649202330B4C1F8A031D1F891
:1002D000A001334A10F0400FF9D0324D0124AA207A
:1002E00055230321C2F80411C2F80C411146C2F88B
:1002F0008450C2F88C00C2F88C30C2F88040C2F83A
:100300008C00C2F88C30D1F88830254A13F0806F09
:10031000F9D00321AA245520C2F88010C2F88C40DD
:100320001146C2F88C00D1F888301D4A13F0407F86
:10033000F9D02324C2F8A440AA2055230124C2F8EE
:10034000AC001146C2F8AC30C2F8A040C2F8AC0014
:10035000C2F8AC30D1F8A830114A13F4806FF9D04C
:100360000321AA235520C2F8A010C2F8AC301146D0
:10037000C2F8AC00D1F8A800094A10F4407FF9D0C7
:100380000949002043F23A03C2F8A801C2F8AC01BF
:10039000C2F8C410C2F8C801136030BC704700BF77
:1003A00000C00F4063000500DE87280430B5254DEE
:1003B000254BD5F8C41083B041F00074C5F8C44093
:1003C000D5F8C420032042F01001C5F8C4101A6803
:1003D000002442F002051D60196821F001021A6034
:1003E0001D6845F0080119601A6822F004051D60B7
:1003F000196841F080421A601D6825F000411960BB
:100400005A6842F001055D605968104D21F0020202
:100410005A6000F095F90822012328604FF4165124
:10042000009400F06FF9012000F08AF9084D4FF4B4
:100430001641286008220123009400F063F903B0FC
:1004400030BD00BF00C00F4000C002400C000010D3
:1004500014000010164A10B5D2F8C410154B41F420
:100460000044C2F8C4401968134841F434021A60C9
:100470005969124C21F480225A61596921F4801281
:100480005A61596921F400125A61596921F4000234
:100490005A6100F05FF900F0EDF92060084800F0C3
:1004A00059F900F0E7F92060FFF780FF002010BD48
:1004B00000C00F4020C00920005A62021000001046
:1004C00000B4C40430B42A4A84B00DF1040C0446CC
:1004D0000D46284B07CAACE803009C428CF800206C
:1004E00029D018DD244B9C421BD003F580418C425F
:1004F00014D104A94D19214B15F80C0CD3F8AC11EB
:10050000820442EA0101C3F8AC11D3F8AC01024005
:10051000C3F8AC2102E01A4884421ED004B030BCBB
:1005200070470DF1100C6544144B15F80C2CD3F8E2
:10053000AC111204E5E704A94D19104B15F80C0C89
:10054000D3F8A811020242EA0101C3F8A811D3F8B6
:10055000A8010240C3F8A821E0E70DF1100C6544A2
:10056000064B15F80C2CD3F8A8119201EBE700BF4D
:1005700008090000000001400080094000C00F4051
:1005800000C000402DE9F047044682B00F46002825
:1005900053D000F06FF9554E554B804630689C4261
:1005A000019000F09C804BDD524B9C425DD003F5E6
:1005B000804294425FD0002302A800EB030E1EF895
:1005C00004CC3F01B8FBFCF3BB422BD2D6F8009021
:1005D000474DDFF820A1AC42CDF8049067D050DC45
:1005E000454B9C4235D000230DF1080E0EEB030C59
:1005F0001CF8041C012920D049082046FFF762FF9F
:100600003268AC4201925ED046DC3B48844226D040
:10061000002302A901EB030E1EF804CCB8FBFCF387
:10062000BB42D8D3E268B3FBF7F342F08001E1604C
:100630002360E06820F08002E26002B0BDE8F0874D
:100640002D498C42B7D12D48D0F8A831C3F381137E
:10065000B2E72A48D0F8A821C2F38113C4E7274A99
:10066000D2F8A811C1F38113D3E72448D0F8AC31F4
:10067000C3F30143A0E7214AD2F8AC11C1F381438F
:100680009AE7544519D01E498C42ACD11B49D1F888
:10069000AC31C3F38143A7E754451AD0184B9C42B1
:1006A000B6D1164BD3F8AC01C0F38143B1E713497F
:1006B000D1F8A831C3F3012396E71048D0F8AC2154
:1006C000C2F3014390E70D4BD3F8A801C0F3012317
:1006D0009FE70A4AD2F8AC11C1F3014399E7074AF0
:1006E000D2F8A811C1F3012366E700BF1409000086
:1006F000000001400080094000C0004000C00F40E1
:1007000000C0094030B4092A9DF808400ED8013BCA
:10071000DDB2053A012D0ED90023072C0ED9002594
:100720009C186419C46030BCFFF72CBF013BDDB2DC
:100730000322012DF0D89B00072CF0D8E500EFE74D
:1007400003289ABF024B53F820000020704700BFD7
:10075000F8080000F0B4404D3F4CD5F80C31D4F807
:100760000C1113F0030F08BF3C4B3B4E01F0030785
:100770000CBF1A6842F21072D6F80C51012F08BF54
:10078000374F05F0030308BF3A68022B08BF354B0B
:10079000314908BF1A68344BB3FBF0F4601EC1F84E
:1007A00004015000012218E0B4FBF0F1CF1F013228
:1007B000B7F5FC7F144622D9B5FBF0F1CD1F01320D
:1007C000B5F5FC7F1BD9B6FBF0F1CD1FA21CB5F52A
:1007D000FC7F14D9E21C212A3BD02349234F244E0D
:1007E0005C18B3FBF0F1DD199E19CF1F03F18E43A6
:1007F00003F5060CB7F5FC7F0CF50C43D4D8541E5A
:10080000154B220401398918AA2455200122C3F866
:100810008410C3F88C401946C3F88C00C3F88020BC
:10082000C3F88C40C3F88C00D1F888000A4A10F055
:10083000806FF9D00321AA205523C2F88010C2F896
:100840008C001146C2F88C30D1F8882012F0407F1D
:10085000FAD0F0BC704700BF00C00F400400001089
:10086000000000100800001000A3E1110046C3239F
:1008700000E9A4351C4A30B4D2F88450D2F8844040
:10088000D2F80411D2F80C3113F0030F04BF174B48
:100890001868154BD3F80C2102F0030C124ABCF176
:1008A000010FD2F80C2108BF114B02F0030C08BF56
:1008B0001868BCF1020F04BF0E4B18680A4BD3F83E
:1008C000802012F0020F0CD0AA04930C5A1C530083
:1008D000C4F307444A1C00FB03F004FB0221B0FBF5
:1008E000F1F030BC704700BF00C00F4004000010A2
:1008F000000000100800001000C00040000001408F
:100900000080094000C0094001010202000000000F
:080910000300000004010208CD
:0C091800001BB70000093D00008000003B
:00000001FF
